:10142400758400852ED2852FD37584018530D285AD
:1014340031D3E4F52FF52E30005730064E855B820C
:10144400855A83E0F52FA3E0F52EA385825B85837F
:101454005AE55B655D700CE55A655C7006755B006A
:10146400755A02855982855883E533F0A3E532F035
:10147400A3858259858358E559655D7014E55865DF
:101484005C700E755900755802800685322E8533BE
:101494002F30010CE52E2534F52EE52F3535F52FAB
:1014A400300210E53F8527F0A4252EF52EE5F03512
:1014B4002FF52F300310E50A852AF0A4252EF52EEA
:1014C400E5F0352FF52F300410E5118529F0A4251A
:1014D4002EF52EE5F0352FF52FE4F531F5303009F2
:1014E4005730054E855B82855A83E0F531A3E0F5DC
:1014F40030A385825B85835AE55B655D700CE55A94
:10150400655C7006755B00755A028559828558833F
:10151400E535F0A3E534F0A3858259858358E55970
:10152400655D7014E558655C700E75590075580258
:10153400800685343085353130080CE5302532F5A8
:1015440030E5313533F531300A10E53F8527F0A415
:101554002530F530E5F03531F531E531C3952C40D2
:0315640003852CD0
:1015670031300B10E50A852AF0A42530F530E5F077
:101577003531F531300C10E5118529F0A42530F50A
:1015870030E5F03531F531300D10E5188528F0A438
:101597002530F530E5F03531F531E531C3952D408E
:1015A70003852D31229016053015031215C230160A
:1015B700031215D23018031215F522E50B2509F58C
:1015C7000BE50C3508F50C93F50A22E512250EF507
:1015D70012E513350DF51393C313F8E5142510F52C
:1015E70014E515350FF51593C31328F51122E519E1
:1015F7002517F519E51A3516F51A93F518227F827E
:1016070085888C8F9295989B9EA1A4A7AAADB0B30D
:10161700B6B9BBBEC1C3C6C9CBCED0D3D5D7D9DC2B
:10162700DEE0E2E4E6E7E9EBEDEEF0F1F2F4F5F601
:10163700F7F8F9FAFBFCFCFDFDFEFEFEFEFEFEFEE2
:10164700FEFEFEFDFDFCFCFBFAFAF9F8F7F6F4F3F3
:10165700F2F0EFEDECEAE8E7E5E3E1DFDDDBD8D632
:10166700D4D1CFCDCAC8C5C2C0BDBAB7B4B2AFAC6A
:10167700A9A6A3A09D9A9794908D8A8784817E7A44
:101687007774716E6B6865625F5C595653504D4A4B
:101697004744423F3C393734322F2D2A282624210C
:1016A7001F1D1B1918161412110F0E0C0B0A080711
:1016B7000605040403020201010000000000000007
:1016C70000000001010202030405060708090A0BCE
:1016D7000D0E1011131516181A1C1E202224272967
:1016E7002B2E303335383A3D404245484B4E515406
:1016F70056595C606366696C6F7275787B7FFEFE16
:10170700FEFEFDFCFCFBFAF8F7F6F4F3F1EFEDEB68
:10171700E9E7E4E2DFDCDAD7D4D0CDCAC6C3BFBC81
:10172700B8B4B0ACA8A39F9B96928D89847F7A7535
:10173700706B66615C57514C47413C37312C262111
:101747001B16100B050000050B10161C21272C3249
:10175700373D42484D53585D62686D72777C81858D
:101767008A8F94989DA1A5AAAEB2B6BABEC1C5C8C4
:10177700CCCFD2D5D8DBDEE1E3E6E8EBEDEFF1F253
:10178700F4F6F7F8F9FBFBFCFDFEFEFEFEFE000C8F
:101797001926333F4C5864707B86919CA6AFB8C11D
:1017A700C9D1D8DEE4EAEFF3F6F9FCFDFEFEFEFD53
:1017B700FCFAF7F4F0EBE6E0DAD4CCC5BCB4ABA1A5
:0E17C700978D83786D61554A3D3125180C00D1
:101ADF00D2F4C2F5C2F675840F85F0C8121F8B744D
:101AEF0003121B2E121F7F7403121B2E121F621262
:101AFF001F627403121B2E121F627402121B2E120E
:101B0F001F627428121B9A7406121B9A740E121BF2
:101B1F009A7401121B9A121F7F7480121B9A22C093
:101B2F0000A2E092F3A2E192F2A2E292F1A2E3927A
:101B3F00F0D2F475840F85F0C8C2F47830D8FE85E2
:101B4F00F0C87830D8FED00022C00075840FA2E410
:101B5F0092F3A2E592F2A2E692F1A2E792F0D2F40A
:101B6F0085F0C8C2F47830D8FE85F0C87830D8FE3A
:101B7F00D00022EF75840FD2F5C2F685F0C8121B84
:101B8F0058121F62121B2E121F622275840FC2F58C
:101B9F00C2F685F0C8121B58121F62121B2E121F9D
:101BAF006222EF14A2E492E6C2E4D2E7121B9A2259
:101BBF00740F121B9A22740D121B9A227F01121B93
:101BCF00B178107F20121B82D8F9227F11121BB11E
:101BDF0078107F20121B82D8F9227F01121BB17857
:101BEF00207F20121B82D8F922C0077F018004C0FA
:101BFF00077F11121BB1D007C082C083C007EF75DA
:101C0F00F010901C29121FA37810E493FF121B826F
:091C1F00A3D8F7D007D083D082CE
:101C280022202020202020202020202020202020AA
:101C38002057414954494E4720464F522052494E59
:101C4800472054454C434F20414E53574552454435
:101C580020205741495420464F5220444953434F6E
:101C68002020205445535420204641494C454420C7
:101C7800202020544553542020504153534544209C
:101C8800202020454550524F4D2054455354202084
:101C980020204155582052454C4159205445535411
:101CA8002020205055534820544F2054414C4B205D
:101CB8002054455354203320434841522F53554212
:101CC80020544553542046495845442053545249BA
:101CD8004E54455354205641524942205354524978
:101CE8004E464143544F52592044454641554C5461
:101CF8002050524F4752414D4D494E47204D4F4479
:101D08004553494D504C455820524550454154453E
:101D1800522020205245434F5244494E472020200C
:011D2800209A
:1028AD0032C28D32758400C2CF32C0E0C083C08287
:1028BD00C0D0C000C0F0C2CFB21A201A2312142407
:1028CD00151BE51B7009751B0A7584017588AF15FD
:1028DD001CE51C7009751C607584027588AF80112C
:1028ED001215AC1536E5367008753604758400D2B0
:1028FD008B758400D2ECD0F0D000D0D0D082D083B4
:10290D00D0E032C2CF32C0E0C0D0C007C000C0831B
:10291D00C08212421975888FD082D083D000D00723
:10292D00D0D0D0E032C0E0C0D0C000C083C082C0E3
:10293D008420121375840F30DF27E5E8540FF5401E
:10294D00D2127541C8801A1541E5417006E540D295
:10295D00E7F54075840F20DF08C212D211D22AD2BA
:10296D002D20141475840F30F828E5E854F0C4F5C3
:10297D0042D2147543C8801A1543E5437006E542EB
:10298D00D2E7F54275840F20F808C214D213D2296C
:10299D00D21C12425E151DE51D702A751D0A1242CC
:1029AD0085151EE51E701E751E0A1242D8151FE5EF
:1029BD001F7012751F061242D91526E52670067571
:1029CD00260A1242E2D084C28DD082D083D000D0AC
:1029DD00D0D0E0323220100DD21085BF3585BE34F7
:0A29ED0075BB01800BC21085BF33DB
:1029F70085BE3275BB00C2ED32C0E0C0D0E544B43D
:102A0700000A054485BE3F75BB07803DB4010A0532
:102A17004485BE3C75BB048030B4020A054485BEBC
:102A27003F75BB068023B4030A054485BE3D75BBCD
:102A3700048016B4040A054485BE3F75BB058009AA
:102A470075440085BE3E75BB04C2EDD0D0D0E032E0
:103C400044313233343536373839302A2341424310
:103C5000202020205354414E44425920202020202F
:103C6000524144494F204F524947494E4154452003
:103C700054454C434F204F524947494E41544520EB
:103C800020202046554E4354494F4E2031202020BD
:103C900020202046554E4354494F4E2032202020AC
:103CA00020202046554E4354494F4E20332020209B
:103CB00020202046554E4354494F4E20342020208A
:103CC00020202046554E4354494F4E203520202079
:103CD00020202046554E4354494F4E203620202068
:103CE00020202046554E4354494F4E203720202057
:103CF00020202046554E4354494F4E203820202046
:103D000020202046554E4354494F4E203920202034
:103D1000202052454345495645204D4F44452020DB
:103D2000205452414E534D4954204D4F444520207C
:103D3000202045204C4541442044454C41592020F9
:103D4000205741495420464F52204D204C45414474
:1042EB001265CF12487775840F1200A41265C312A2
:1042FB005F09125F4212623B12567E20A503120E1B
:10430B00DA9000A5E4F020A432302915C229E54249
:10431B00540FFFEF903C4093FF90008CEFF0124D49
:10432B005C302AE2C22AE540540FFFEF903C4093E9
:10433B00FF90008BEFF0124E3F80CB9000A5E0FF7B
:10434B00EF12401C437400437901437E0243830305
:10435B00438804438D05439306439907439F0843C2
:10436B00A50943AB0A00004311125A058098124469
:10437B00758093125488808E1262688089122A5736
:10438B008084122D98024311124DCE024311125DFF
:10439B006D0243111258E2024311126415024311CC
:0A43AB00124992024311024311224D
:105A05001263FB1265B71265C31264CD1261B01241
:105A1500623B125AD81266859000ACE4F09000B152
:105A2500E4F09000A6E4F09000EEE4F09000EDE4E0
:105A3500F07BFF7A3C7950126124121BDA753832FB
:075A45009000A5E004F0222F
:10447500E53860030245331246961251FC302B0B8A
:1044850012630BC22B9000A5E4F022301F0B125FC4
:104495007BC21F9000A5E4F0221264975040900063
:1044A500E1E0FF9000A7EFF09000EBE0FFEFB40232
:1044B500031265B19000ECE0FFEFB402031265BD95
:1044C5009000B1E4F07BFF7A3C79701261247BFFA8
:1044D5007A3D79301261559000A57402F02212647C
:1044E500A9EF604A9000EAE0FFEF60421264DD90B8
:1044F50000E2E0FF9000A8EFF09000EBE0FFEFB4E2
:1045050002031265B19000ECE0FFEFB402031265FF
:10451500BD9000B1E4F07BFF7A3C79601261247BA9
:0F452500FF7A3D79401261559000A57406F0228F
:105488001223549000A7E0FFEF702D1264DD900006
:10549800EBE0FFEFB402031265B19000ECE0FFEF20
:1054A800B402031265BD75370A7BFF7A3D79101285
:1054B80061559000A57403F0124696302B0B1263C9
:1054C8000BC22B9000A5E4F022301F0A125F7BC2AA
:0754D8001F9000A5E4F02283
:10626800122354E537702312666D12663A1263FBE7
:106278009000D8E0FF9000A3EFF09000EDE4F090DC
:0B62880000EEE4F09000A57405F02289
:102A570020A6031250CC1266371223541217D51230
:102A67004F8D1251FC123D501246969000EEE0FF3A
:102A7700EF603F1263FB1264CD9000EBE0FFEF6461
:102A87000160099000EBE0FFEFB402031265B79015
:102A970000ECE0FFEF640160099000ECE0FFEFB4A9
:102AA70002031265C39000EF740AF09000A5740941
:102AB700F0229000DBE0FFEF705C9000A6E0FFEFF4
:102AC700602B900098E0FFEF70239000A6E4F09051
:102AD7000099E4F09000DEE0FF9000D9E0FEEE2FD1
:102AE700FF9000A1EFF09000A5740AF022900098E3
:102AF700E0FFEF702190009CE0FFEF70199000DE7F
:102B0700E0FF9000D9E0FEEE2FFF9000A1EFF090DC
:102B170000A5740AF0229000DBE0FFEFB4012190DA
:102B27000098E0FFEF70199000DEE0FF9000D9E019
:102B3700FEEE2FFF9000A1EFF09000A5740AF0229F
:102B47009000DBE0FFEFB4022190009CE0FFEF7004
:102B5700199000DEE0FF9000D9E0FEEE2FFF900015
:102B6700A1EFF09000A5740AF0229000DBE0FFEFE0
:102B7700D3940240219000B1E0FFEF70199000DE7E
:102B8700E0FF9000D9E0FEEE2FFF9000A1EFF0905C
:102B970000A5740AF022302B201263FB1265B712CE
:102BA70065C31264CD12630BC22B12665812665EA0
:102BB70012663A9000A5E4F022301F1D1263FB1243
:102BC70065B71265C312665812665E12663A125FDF
:102BD7007BC21F9000A5E4F0221264974018900072
:102BE700DEE0FF9000D9E0FEEE2FFF9000A1EFF0AE
:072BF7009000A57408F02214
:102D980020A6031250CC12650C1263591223541248
:102DA80017D512665E126658124F8D1251FC123DED
:102DB800501246969000EEE0FFEF603F1263FB1260
:102DC80064CD9000EBE0FFEF640160099000EBE058
:102DD800FFEFB402031265B79000ECE0FFEF640167
:102DE80060099000ECE0FFEFB402031265C39000A5
:102DF800EF740AF09000A57409F0229000DBE0FF60
:102E0800EF701A900098E0FFEF700E90009CE0FFC2
:102E1800EF600A1264A9EF7004125A93229000DB43
:102E2800E0FFEFB4010C900098E0FFEF6004125A45
:102E380093229000DBE0FFEFB4021290009CE0FFC9
:102E4800EF600A1264A9EF7004125A93229000DB13
:102E5800E0FFEFB4030C9000B1E0FFEF6004125AFA
:102E680093229000DBE0FFEFB4040C9000B1E0FF88
:102E7800EF6004125A9322302B201263FB1265B7BD
:102E88001265C31264CD12667012630B1266581273
:102E98006670C22B9000A5E4F022301F1D1263FB60
:102EA8001265B71265C312665812663A1266701236
:102EB8005F7BC21F9000A5E4F02212649740401285
:102EC80064CD1263FB9000EBE0FFEF6401600990B2
:102ED80000EBE0FFEFB402031265B79000ECE0FFEF
:102EE800EF640160099000ECE0FFEFB402031265A3
:102EF800C312665812665E12663A9000A5E4F02284
:104DCE001251FC1264A9EF600A9000E2E0FF90001D
:104DDE00A8EFF09000A8E0FFEF70299000E2E0FF4E
:104DEE00EF60211264CD9000EBE0FFEFB4020312EE
:104DFE0065B79000ECE0FFEFB402031265C39000BC
:104E0E00A5E4F022126497500975370A9000A57434
:104E1E0007F0124696302B0B12630BC22B9000A597
:104E2E00E4F022301F0A125F7BC21F9000A5E4F04F
:014E3E002251
:105D6D00126497400375370AE537701275370A7B51
:105D7D00FF7A3D79101261559000A57403F012461B
:105D8D0096302B0B12630BC22B9000A5E4F0223042
:0D5D9D001F0A125F7BC21F9000A5E4F022D8
:1058E2009000A1E0FFEF70401264CD1263FB9000C4
:1058F200EBE0FFEF640160099000EBE0FFEFB40220
:10590200031265B79000ECE0FFEF640160099000BC
:10591200ECE0FFEFB402031265C312665812665E32
:0959220012663A9000A5E4F0229F
:106415009000EFE0FFEF700E12665812665E12668E
:076425003A9000A5E4F0220B
:104992009000A1E0FFEF70041260ED221266371260
:1049A20023541217D5123D50124696302B0B126328
:1049B2000BC22B9000A5E4F022301F0B125F7BC2CA
:1049C2001F9000A5E4F0229000EEE0FFEF603E129F
:1049D20063FB1264CD9000EBE0FFEF64016009908D
:1049E20000EBE0FFEFB402031265B79000ECE0FFCA
:1049F200EF640160099000ECE0FFEFB4020312657E
:0E4A0200C39000EF740AF09000A57409F02232
:105A9300126670126688125A4C12663A9000E8E059
:105AA300FFEF60069000AE7401F01263E19000EB2B
:105AB300E0FFEFB401031265B19000ECE0FFEFB437
:105AC30001031265BD7BFF7A3D7920126155900079
:055AD300A57404F0229F
:1060ED007BFF7A3D791012615512663A12666D1278
:1060FD0063FB9000EBE0FFEFB401031265B7900076
:10610D00ECE0FFEFB401031265C39000A57405F038
:01611D00225F
:1064CD009000E0E0FFEF60041265C9221265CF2253
:1064DD009000E0E0FFEF60041265CF221265C92243
:106497009000DFE0FFEF60061265F9B32222126574
:0264A700F922D8
:103E5100900091E0FF703B9000CAE060159000CBAC
:103E6100E0FEE53ED39E40249000CCE0900093021A
:103E71003F099000CBE0FEE53EC39E500F9000CC81
:103E8100E0900093F09000917403F022E49000948C
:103E9100F022EF640170249000CBE024FBFFE53EAB
:103EA100D39F406C900093E06003023F4C900094DC
:103EB10004F09000CDE0900092804D900091E0FFE1
:103EC100B402179000CBE024FBFEE53ED39E4002F6
:103ED100805F900092E070738066EF6403703390AE
:103EE10000CBE02405FFE433FEC3E53E9FEE648092
:103EF100F8748098501A900093E0704F90009404E9
:103F0100F09000CDE0900092F0900091E004F0225A
:103F11008034900091E06404702C9000CBE0240583
:103F2100FFE433FEC3E53E9FEE6480F87480985051
:103F3100099000CDE0900092F022900092E0700B89
:0C3F4100900094F08001E4900091F022C8
:10519B00900091E0700E1265D550559000CCE090C8
:1051AB000093801E900091E0B401221265D5501A35
:1051BB00900093E0701790009404F09000CDE09075
:1051CB000092F0900091E004F022E4801F90009197
:1051DB00E0B4021C1265D550099000CDE09000920E
:1051EB00F022900092E07008900094F0900091F003
:0151FB002291
:0D650C009000C9E0600302519B123E512235
:103D5000900095E0FF703B9000CEE060159000CFA2
:103D6000E0FEE53DD39E40249000D0E09000970215
:103D70003E109000CFE0FEE53DC39E500F9000D076
:103D8000E0900097F09000957403F022E490009882
:103D9000F022EF640170259000CFE024FBFFE53DA9
:103DA000D39F4074900097E0701290009804F090B8
:103DB00000A6F09000D1E09000968054900095E02D
:103DC000B402179000CFE024FBFFE53DD39F4002F3
:103DD0008064900096E07002806B900095E0FF6434
:103DE0000370379000CFE02405FDE433FCE53DC3CC
:103DF0009DEC6480F8748098501E900097E0701AD3
:103E000090009804F09000A6F09000D1E090009609
:103E1000F0900095E004F0228031EF6404702C9063
:103E200000CFE02405FFE433FEC3E53D9FEE648050
:103E3000F874809850099000D1E0900096F022909C
:103E40000096E07006900098F08001E4900095F0F4
:013E5000224F
:104F8D00900099E070191265E1500E9000D4E090F8
:104F9D00009BF0900099E004F0E490009CF02290CA
:104FAD000099E0B401221265E1501A90009BE07067
:104FBD001790009C04F09000D5E090009AF09000BE
:104FCD0099E004F022E4801F900099E0B4021C12D5
:104FDD0065E150099000D5E090009AF02290009A7A
:0C4FED00E0700890009CF0900099F02209
:1051FC0090009DE0700E1265DB50559000D2E0904F
:10520C00009F801E90009DE0B401221265DB501AB5
:10521C0090009FE070179000A004F09000D3E090F5
:10522C00009EF090009DE004F022E4801F90009D11
:10523C00E0B4021C1265DB50099000D3E090009E94
:10524C00F02290009EE070089000A0F090009DF07D
:01525C00222F
:1064A9009000D7E060069000A0E0FF22900094E001
:0264B900FF22C0
:106359009000D8E0FF601D90009CE070069000A0BE
:10636900E060069000A3EFF0229000A3E070059092
:05637900009004F02279
:104CE90054564F582020434F53202053454E534587
:104CF900004F4E202020202020202020202020206E
:104D090020004F464620202020202020202020203F
:104D1900202000191823A01296203D129623A012D4
:104D29009627631488203D148823A01488276316C6
:104D3900B8203D16B823A016B827631918203D19C5
:104D490018276312962B8C14882B8C16B82B8C1968
:034D5900182B8C88
:104877001266131266101265D5E433F54F126616E9
:10488700E433F54F126619E433F54F12661CE4332F
:10489700F54F12661FE433F54F126622E433F54FE6
:1048A700126625E433F54F126628E433F54F126696
:1048B7002BE433F54F1265E7E433F54F12662EE428
:1048C70033F54F1265F3E433F54F12663112663450
:1048D70012663D1266401266431266461266491218
:1048E700664C12664F126652126661126664126651
:1048F7006712666A12667312667612667912667CAA
:0649070012667F026682C9
:0665B10075840FD2FC22EC
:0665B70075840FC2FC22F6
:0665BD0075840FD2B72225
:0665C30075840FC2B7222F
:0665C90075840FD2FE22D2
:0665CF0075840FC2FE22DC
:1063E10075840FD2FD9000EBE0B401031265B1900A
:0A63F10000ECE0B401031265BD22C8
:1063FB0075840FC2FD9000EBE0B401031265B790FA
:0A640B0000ECE0B401031265C322A7
:03661000C2932210
:03661300D29322FD
:0665D50075840FA2FA22FA
:03661600A2A0221D
:03661900A2A12219
:03661C00A2A22215
:03661F00A2A32211
:03662200A2A4220D
:03662500A2A52209
:03662800A2A62205
:03662B00A2A72201
:0665DB0075840FA2F922F5
:0665E10075840FA2DD220B
:0665E70075840FA2DE2204
:03662E00A2922213
:0665ED0075840FA2DA2202
:0665F30075840FA2DB22FB
:0665F90075840FA2DC22F4
:0665FF0075840FA2D822F2
:0666050075840FA2D922EA
:03663100D208226A
:03663400C2082277
:03663700D2092263
:03663A00C2092270
:03663D00D20A225C
:03664000C20A2269
:03664300D202225E
:03664600C202226B
:03664900D20B224F
:03664C00C20B225C
:03664F00D20C2248
:03665200C20C2255
:03665500D20D2241
:03665800C20D224E
:03665B00D2182230
:03665E00C218223D
:03666100D20E2234
:03666400C20E2241
:03666700D20F222D
:03666A00C20F223A
:03666D00D2002236
:03667000C2002243
:03667300D201222F
:03667600C201223C
:03667900D2032227
:03667C00C2032234
:03667F00D2042220
:03668200C204222D
:105A4C00E4FDFCED25E0FFEC33FE74002FF58274D1
:105A5C00023EF583E4F0A3F00DBD00010CBC0EE397
:105A6C00BDE0E07558027559007402F55AF55B906B
:105A7C0000D9E075F0BEA4AEF02400F55DEE340262
:065A8C00F55CC200D2052A
:015A920022F1
:03668500C2052229
:105AD800E4FDFCED25E0FFEC33FE74002FF5827445
:105AE800023EF583E4F0A3F00DBD00010CBC0EE30B
:105AF800BDE0E07558027559007402F55AF55B90DF
:105B080000D9E075F0BEA4AEF02400F55DEE3402D5
:045B1800F55CD20660
:015B1C002266
:03668800C2062225
:0B65490075081575095ED215D20322FB
:0B65540075081575095ED215D20B22E8
:0765A300C215C203C20B2266
:0B655F009000BD123073D216D204224F
:0B656A009000BE123073D216D20C223B
:0C307300E0F529E4F512F513F514F5154D
:10307F00EF12401C317A2331692A30B73030C93111
:10308F0030DB3230ED3330FF34311135312336310F
:10309F003537314738315839318B41319C4231AD59
:1030AF004331BE44000031D6904D1CE493F50D74AE
:1030BF000193F50E904D1E0231CD904D20E493F506
:1030CF000D740193F50E904D220231CD904D24E4F5
:1030DF0093F50D740193F50E904D260231CD904D61
:1030EF0028E493F50D740193F50E904D2A0231CD1E
:1030FF00904D2CE493F50D740193F50E904D2E0227
:10310F0031CD904D30E493F50D740193F50E904D44
:10311F00320231CD904D34E493F50D740193F50ED9
:10312F00904D360231CD904D38E493F50D740193E7
:10313F00F50E904D3A0231CD904D3CE493F50D7460
:10314F000193F50E904D3E8075904D40E493F50D33
:10315F00740193F50E904D428064904D44E493F5C5
:10316F000D740193F50E904D468053904D48E493A6
:10317F00F50D740193F50E904D4A8042904D4CE43D
:10318F0093F50D740193F50E904D4E8031904D5087
:10319F00E493F50D740193F50E904D528020904DF0
:1031AF0054E493F50D740193F50E904D56800F90E6
:1031BF004D58E493F50D740193F50E904D5AE49329
:0831CF00F50F740193F51022C5
:0765AA00C216C20CC204225C
:05660B00C215C20322CC
:0B6575007508027509ABD215D20B228D
:0B65800075081A7509ABD215D20B226A
:1050CC00124F8D1251FC7BFF7A4C79E912612490BE
:1050DC00009CE07BFF60067A4C79FA80047A4D796B
:1050EC000B1261557F17121BB1AF3E121FE89000D7
:1050FC006CE0FF121B8290006DE0FF121B8290008F
:10510C006EE0FF121B827F1C121BB1AF3D121FE819
:10511C0090006CE0FF121B8290006DE0FF121B826E
:08512C0090006EE0FF021B82FF
:10024D0020202020202020202020202020202020A1
:10025D002020202020202020202020202020202091
:10026D002054454C434F2050524F4752414D202072
:10027D0020524144494F2050524F4752414D20206A
:10028D002050484F4E452050524F4752414D20204F
:10029D0020434F4D50552050524F4752414D202035
:1002AD00202041434345535320434F4445202020B4
:1002BD0044544D462054454C434F204C4556454CD7
:1002CD0044544D4620524144494F204C4556454CCF
:1002DD004245455020524144494F204C4556454CCE
:1002ED00424545502054454C434F204C4556454CB6
:1002FD0054454C434F20524144494F204C45564C98
:10030D00524144494F2054454C434F204C45564C87
:10031D00524144494F204C494D4954204C45564C6F
:10032D002045494120544F4E45204C4556454C20C3
:10033D004C4F57204755415244204C4556454C2073
:10034D0048494748204755415244204C4556454C55
:10035D00564F494345205241444930204C45564C57
:10036D00564F4943452054454C434F204C45564C20
:10037D0020434F53204F5220535155454C43482055
:10038D002020434F5320504F4C4152495459202067
:10039D00434F53205452494747455220564F4C54D2
:1003AD00434F5320414351554953542054494D45D2
:1003BD00434F532052454C454153452054494D45DB
:1003CD002053454E534520504F4C415249545920CE
:1003DD0053454E205452494747455220564F4C5491
:1003ED0053454E20414351554953542054494D4591
:1003FD0053454E2052454C454153452054494D459A
:10040D005220564F582041435155495354494F4E50
:10041D0020525820564F582052454C4541534520A7
:10042D005420564F582041435155495354494F4E2E
:10043D0020545820564F582052454C454153452085
:10044D00204F5045524154494E47204D4F44452071
:10045D0020564F58204F5220434152524945522069
:10046D002020564F58204143544956495459202075
:10047D00202054454C434F2044454C4159202020C9
:10048D002020524144494F2044454C4159202020C1
:10049D0053454E53452C20564F582C20544F4E4506
:1004AD0020204143434553532044454C415920207E
:1004BD00205455524E204F4E2044454C415920203A
:1004CD00205455524E204F46462044454C4159200C
:1004DD004449474954414C20494E20504F4C4152BC
:1004ED00434E544C2052454C415920504F4C415293
:1004FD002020452D44454C41592050425820202064
:10050D002020452D44454C41592052454320202063
:10051D00202052494E474F5554204D4F44452020E1
:10052D00414E535745522052494E47204E4D42524F
:10053D0020202052494E4720535041434520202032
:10054D00202052494E4720414E53574552202020DE
:10055D0052494E47205452414E534954494F4E53E0
:10056D0045494120544F4E4520454E41424C452072
:10057D0046554E4354494F4E20382053454C454324
:10058D00524144494F2053454C454320454E424C22
:10059D00204155582052454C4159204D4F4445203E
:1005AD002043542052454C4159204D4F4445202065
:1005BD00202020202020202020202020202020202E
:1005CD00202020202020202020202020313D454E9D
:1005DD002020202020202020202020524154494F2F
:1005ED002020202020202020202020303D434F534C
:1005FD002020202020202020202020313D504F532E
:10060D0020202020202020202020202031204D536C
:10061D0020202020202020202020203130204D534C
:10062D0020202020202020202020313030204D532C
:10063D002020202020202020202020202053454332
:10064D00202020202020202020202020204D494E19
:10065D002020202020202020202020204D4F4445E8
:10066D002020202020202020202020313D564F58B2
:10067D00202020202020202020202052494E47538A
:10068D0020202020202020202020204359434C458D
:10069D0020202020202020202020313D544F4E4569
:1006AD002020202020202020504F4C4152495459C9
:1006BD008201001102381500018201011103381564
:1006CD000001820102110438150001820103110598
:1006DD003815000178060411060119000082030A7D
:1006ED001107391500FF82030B1108391500FF8220
:1006FD00030C1109391500FF82030D110A3915007C
:10070D00FF82030E110B391500FF82030F110C39F7
:10071D001500FF820310110D391500FF8203111111
:10072D000E391500FF820312110F391500FF8203D8
:10073D00131110391500FF8203141111391500FF23
:10074D008203151112391500FF82011611133A1586
:10075D00000182011711143B1500018203181115B8
:10076D00391500FF82021911163C15006382021A19
:10077D0011173D15006382011B11183B15000182F5
:10078D00031C1119391500FF82021D111A3C1500A9
:10079D006382021E111B3D15006382021F111C3C5A
:1007AD00150063820220111D3E1500638202211186
:1007BD001E3C150063820222111F3E15006382014B
:1007CD00231120411500028201241121421500013F
:1007DD0082022511224015006382022611233D1548
:1007ED00002882022711243D150028820128112599
:1007FD004115000482022911263E150A6382022A40
:10080D0011273C15006382022B11283D15006382D0
:10081D00012C11294615000182012D112A461500C2
:10082D000182022E112B3D1501FF82022F112C3E4C
:10083D00150063820130112D3C150001820131112B
:10084D002E43150009820232112F3C1500638201DF
:10085D00331130411500018203341131441501FF6C
:10086D0082013511323815000182013611334515DB
:10087D00000182013711343815000182013811351C
:10088D004115000382013911364115000320202046
:10089D002020202020202020202020202082010127
:1008AD0011020C15000120202020202020202020C6
:1008BD0020202020202082010111020C1500012092
:1008CD0020202020202020202020202020202064D7
:1008DD0001001102091500012020202020202020D8
:1008ED0020202020202020200101010101010101F3
:1008FD0001000000000000000000000000000000EA
:10090D0000000000000000000000000000000000DA
:10091D0000000000000000000000000000000000CA
:10092D0000000000000000000000000000000000BA
:10093D0000000000000000000000000000000000AA
:10094D0000002020202020202020202020202020DA
:10095D002020010101010101010101000000000041
:10096D00000000000000000000000000000000007A
:10097D00000000000000000000000000000000006A
:10098D00000000000000000000000000000000005A
:10099D00000000000000000000000000000000004A
:1009AD0000000000000000000000000020202020BA
:1009BD0020202020202020202020202001010101A6
:1009CD000101010101000000000000000000000015
:1009DD00000000000000000000000000000000000A
:1009ED0000000000000000000000000000000000FA
:1009FD0000000000000000000000000000000000EA
:100A0D0000000000000000000000000000000000D9
:100A1D000000000000002020202020202020202089
:100A2D0020202020202082010011021E150001012E
:100A3D00010101313233343536FF323232FFFFFFDF
:100A4D00550CFF3232000180000A0080000A000AB6
:100A5D00000A0001002828001E140000012863016F
:100A6D000163000A01010102000000000000000006
:100A7D0044313233343536373839302A2341424305
:100A8D0044AAA3C1C2C3C4D7ABA8A92A23414243D8
:100A9D0036333036373036393437313937343437F9
:100AAD0037303739373832353835343838353931DC
:100ABD0035393438393734313030313033313037EE
:100ACD0031313031313431313831323331323731F6
:100ADD0033313133363134313134363135313135DD
:100AED0036313539313632313635313637313731B8
:100AFD0031373331373731373931383331383631A2
:100B0D003839313932313936313939323033323091
:100B1D003632313032313832323532323932333396
:100B2D003234313235303235343030363030373092
:100B3D003135303137303231303233303235303289
:100B4D00363033313033323033363034333034376E
:100B5D003035303035313035333035343036353061
:100B6D00373130373230373330373431313431314A
:100B7D003531313631323231323531333131333243
:100B8D00313334313431313433313435313532312F
:100B9D00353531353631363231363531373231370B
:100BAD003432303532313232313432323332323511
:100BBD0032323632343332343432343532343632F2
:100BCD0035313235323235353236313236333236E1
:100BDD0035323636323731323734333036333131D0
:100BED0033313533323533333133333233343333C9
:100BFD0034363335313335363336343336353337A2
:100C0D0031343131343132343133343233343331B0
:100C1D003433323434353434363435323435343487
:100C2D00353534363234363434363534363635306F
:100C3D00333530363531363532333532363533326C
:100C4D003534363536353630363631323632343651
:100C5D003237363331363332363534363632363640
:100C6D00343730333731323732333733313733323C
:100C7D0037333437343337353441424344454647AF
:100C8D0048494A4B4C4D4E4F50515253545556575F
:100C9D0058595A6162636465666768696A6B6C6D01
:100CAD006E6F707172737475767778797A303132C0
:100CBD0033343536373839607E21402324255E267E
:100CCD002A28295F2D2B3D7B7D5B5D7C3A3B3C3E8D
:100CDD002C2E3F2F202020202020202020202020BF
:100CED0020474C4F42414C202020202020204354AF
:100CFD0043535320434F444520202020202020449F
:100D0D00435320434F44452020202020204C545253
:100D1D0020524550454154455220202020535045E6
:100D2D004544204449414C494E47202020535045CD
:100D3D0045442043414C4C494E47202020205054DF
:100D4D0043204E554D424552202020202020564F05
:100D5D00494345204D455353414745532020564F58
:100D6D0049434520504C41594241434B2020204995
:100D7D004E56414C49442054595045202020204F77
:100D8D005554204F462052414E4745202020494C76
:100D9D004C4547414C2056414C554520204D55530F
:100DAD00542046494C4C204649454C44202020496E
:100DBD004C4C4547414C20434F4445202020444155
:100DCD00544120414343455054454420204C494E05
:100DDD0045204E554D4245523A2020202055534531
:100DED00522050524F4752414D4D494E4755534554
:100DFD00522049443A2020202020202020564F49BF
:100E0D004345205245434F5244494E472020494CBB
:100E1D004C4547414C20454E545259202020494CB9
:100E2D004C4547414C2047414E4720202020202053
:100E3D00434F4D504C455445442020202020474CD5
:100E4D004F42414C20454550524F4D2020202043CC
:100E5D005443535320454550524F4D2020202020C0
:100E6D0044435320454550524F4D202020202020F3
:100E7D004C545220454550524F4D2020202044497E
:100E8D00414C494E4720454550524F4D202043413E
:100E9D004C4C494E4720454550524F4D2020202067
:100EAD0050544320454550524F4D2020202052454F
:100EBD0050454154455220454550524F4D202049F3
:0D0ECD004E495449414C495A494E47202096
:105F7B009000A47464F0E4900000F030200B301F0C
:105F8B0024125C2C12215B80F530210B301F161272
:105F9B005C6E12215B80F530220B301F0812254CF2
:065FAB0012215B80F522CB
:10215B009000A4E07012900000E0D394004009C2FC
:10216B0020C221C222C21F22900000E012401C227A
:10217B007400227701227A02227D032280042282BC
:10218B0005228406228607228908228C0A228F0BBD
:10219B0022920F229510229814229B15229E19220F
:1021AB00A11A22A41B22A71E22AA1F22AD2322B0F2
:1021BB002422B32822B62922B92D22BC2E22BF2FCE
:1021CB0022C23022C53222C83322CA3422CD352254
:1021DB00D06422D36522D66622D96722DC6E22DE3A
:1021EB006F22E07023227122E27822E47922E67AD0
:1021FB0023227B22E88222EA8322EC8422EE8522B0
:10220B00F18C22F48D22F68E22F88F22FB9622FE81
:10221B00972300982302992305A02308A1230BA23F
:10222B00230DA32310AA2312AB2315AC2317AD2325
:10223B001AB4231DB52320B62322B72324BE23278C
:10224B00BF232AC0232DC12322C22333F02336F10F
:10225B002339F2233CFA233FFB2342FC2345FD2386
:10226B0048FE234BFF0000234E0264BB0263C202F5
:10227B005B1D0262BD800480028000025898022F11
:10228B00080260860231D702553502332502558983
:10229B00023473025CB00252BD0239AB02571D020D
:1022AB0035C102576902370F0257B502385D02611B
:1022BB00DF025ED002592B12584D0253D48000021C
:1022CB004F1F025BE90255DD025B61025FB10254F5
:1022DB002E80468032804B80408022804580078054
:1022EB0026803F0258010243B5801C803502562ED2
:1022FB00024A108008802B025CEF0245E6024EB0CA
:10230B0080200245348012024B868016023AF60278
:10231B004B0A025063800B800C024BFF0256CE021D
:10232B004742025DAA0254DF0262E4024FF90264E3
:10233B00ED025378026694026695026696024A8D08
:09234B00026697E4900000F02204
:1064BB00E4900002F09000A47464F0900000E004FB
:0264CB00F022BD
:1063C200121BCB121BDA7BFF7A0D79EA1261247F52
:0F63D20011121BB1C226C223900000E004F0227A
:105B1D00302340900001E0FFC223BF2A0790000010
:105B2D00E004F022EF6423702A7F23121B82900081
:105B3D0002E004F0E0C394034013C220C221C2224C
:105B4D00C21FE4900000F0126293021BE990000066
:035B5D007402F0DF
:015B60002222
:1062BD007BFF7A0D79EA126124121BDA7F11121B12
:1062CD00B1126519E490003CF07F2A121B82C226A0
:0762DD00900000E004F02234
:10589800302346900001E0F55EC223E55E642A608D
:1058A80038AF5E1264FD5022AF5E121B8290003C3E
:1058B800E02403F582E43400F583E55EF090003CD3
:1058C800E004F0900000E004F0227BFF7A0E791AE1
:0958D80012612490000074FAF042
:0158E10022A4
:102F0800202303023072900001E0FFC223BF2A078A
:102F18009000007403F022EF642360030230631210
:102F28001B82900004E064397077A3E06439707103
:102F3800A3E06439706BD227900003E0FFB4310836
:102F4800E4900036F0022FD2EFB43208E490003754
:102F5800F0022FE5EFB43302803E900003E0FFB4A7
:102F68003408E4900038F0023013EFB43508E490E8
:102F78000039F0023029EFB43608E490003AF00244
:102F8800303FEFB437028010900003E0B43802807D
:102F980007900003E0B4390B7BFF7A0E792A0230E0
:102FA80069C227900003E0FFB43016A3E0B43011E3
:102FB800A3E0B4300CA3E0B43007900000740AF02A
:102FC80022EFB4310C12531B5007900000740FF01D
:102FD80022900003E0B4320C12525D5007900000BA
:102FE8007414F022900003E0B43311A3E0B4300C61
:102FF8001263A150079000007419F022900003E0BA
:10300800B4340FA3E0B4300A126443900000741E75
:10301800F022900003E0B4350FA3E0B4300A126444
:10302800589000007423F022900003E0B4360FA3F8
:10303800E0B4300A12646D9000007428F022900009
:1030480003E0B43716A3E0B43011A3E0B4300CA306
:10305800E0B43007900000742DF0227BFF7A0E79DF
:0A3068001A12612490000074FAF0BF
:01307200223B
:1060860090003B740BF090003C7407F0E4900049DC
:10609600F090004A743AF0E490004BF07BFF7A0CE3
:1060A60079EA12612412614F7F1E121BB190000023
:0460B6007432F0222E
:1031D700124C74D3900072E09434900071E0940024
:1031E700400A12611E90000074FAF022900071E00C
:1031F700FEA3E0FF9006BD75F009124010EE75F0D2
:1032070009A42583F583E493900040F09006BE75EA
:10321700F009EF124010EE75F009A42583F583E459
:1032270093900041F0900071A3E09006BF75F009FC
:10323700124010EE75F009A42583F583E4939000FE
:1032470042F09006C075F009EF124010EE75F009D4
:10325700A42583F583E493900043F0900071A3E0E5
:103267009006C175F009124010EE75F009A4258388
:10327700F583E493FD900044F09006C275F009EFE2
:10328700124010EE75F009A42583F583E4939000AE
:1032970045F0900071A3E09006C375F00912401045
:1032A700EE75F009A42583F583E493900046F0902A
:1032B70006C475F009EF124010EE75F009A42583D6
:1032C700F583E493900047F0900071A3E09006C562
:1032D70075F009124010EE75F009A42583F583E413
:1032E70093900048F0ED6015900044E075F010A44D
:1032F700244DF9740235F0FA7BFF126124900045E2
:10330700E0FF601175F010A4244DF9740235F0FA4E
:0E3317007BFF126155900040E0900000F02214
:1055350090003B7410F090003C7407F090004974A3
:105545003AF0E490004AF0900036E090004BF07B92
:10555500FF7A0C79FA12612412614F7F0D121BB18B
:10556500900004E0FF121B82900005E0FF121B82F1
:10557500900006E0FF121B827F1E121BB1900000F7
:045585007432F0226A
:10332500124C74D3900072E09400900071E0940008
:10333500400A12611E90000074FAF022900071E0BC
:10334500FEA3E0FF9008AA75F009124010EE75F093
:1033550009A42583F583E493900040F09008AB75AC
:10336500F009EF124010EE75F009A42583F583E40A
:1033750093900041F0900071A3E09008AC75F009BE
:10338500124010EE75F009A42583F583E4939000AF
:1033950042F09008AD75F009EF124010EE75F00996
:1033A500A42583F583E493900043F0900071A3E096
:1033B5009008AE75F009124010EE75F009A425834A
:1033C500F583E493FD900044F09008AF75F009EFA4
:1033D500124010EE75F009A42583F583E49390005F
:1033E50045F0900071A3E09008B075F00912401007
:1033F500EE75F009A42583F583E493900046F090DB
:1034050008B175F009EF124010EE75F009A4258397
:10341500F583E493900047F0900071A3E09008B223
:1034250075F009124010EE75F009A42583F583E4C3
:1034350093900048F0ED6015900044E075F010A4FD
:10344500249AF9740835F0FA7BFF1261249000453F
:10345500E0FF601175F010A4249AF9740835F0FAAC
:0E3465007BFF126155900040E0900000F022C5
:1055890090003B7415F090003C7407F0900049744A
:105599003AF0E490004AF0900037E090004BF07B3D
:1055A900FF7A0D790A12612412614F7F0C121BB127
:1055B900900004E0FF121B82900005E0FF121B829D
:1055C900900006E0FF121B827F1E121BB1900000A3
:0455D9007432F02216
:10347300124C74D3900072E09400900071E09400B9
:10348300400A12611E90000074FAF022900071E06D
:10349300FEA3E0FF9008C375F009124010EE75F02B
:1034A30009A42583F583E493900040F09008C47544
:1034B300F009EF124010EE75F009A42583F583E4BB
:1034C30093900041F0900071A3E09008C575F00956
:1034D300124010EE75F009A42583F583E493900060
:1034E30042F09008C675F009EF124010EE75F0092E
:1034F300A42583F583E493900043F0900071A3E047
:103503009008C775F009124010EE75F009A42583E1
:10351300F583E493FD900044F09008C875F009EF3B
:10352300124010EE75F009A42583F583E49390000F
:1035330045F0900071A3E09008C975F0091240109E
:10354300EE75F009A42583F583E493900046F0908B
:1035530008CA75F009EF124010EE75F009A425832F
:10356300F583E493900047F0900071A3E09008CBBB
:1035730075F009124010EE75F009A42583F583E474
:1035830093900048F0ED6015900044E075F010A4AE
:1035930024B3F9740835F0FA7BFF126124900045D7
:1035A300E0FF601175F010A424B3F9740835F0FA44
:0E35B3007BFF126155900040E0900000F02276
:105CB0007BFF7A0D791A1261247BFF7A0D79FA1233
:105CC00061557F0E121BB1900005E0FF121B829000
:105CD0000006E0FF121B827F1A121BB190003B747A
:0F5CE0001AF090003C7404F09000007432F0222F
:1052BD003028079000007403F02212614F7F1E12F8
:1052CD001BB1125134900073E0FEA3E0FFD39400A4
:1052DD00EE9400402FEF94FBEE9400502790003B8E
:1052ED00741BF090003C7407F0900049743AF0E4A0
:1052FD0090004AF0900035E01490004BF0900000C3
:0E530D007432F02212611E90000074FAF02239
:1039AB00D3900072E09400900071E09400400A12F2
:1039BB00611E90000074FAF022900071E0FEA3E00B
:1039CB00FF9008DC75F009124010EE75F009A42584
:1039DB0083F583E493900040F09008DD75F009EFD8
:1039EB00124010EE75F009A42583F583E493900043
:1039FB0041F0900071A3E09008DE75F009124010C1
:103A0B00EE75F009A42583F583E493900042F090C2
:103A1B0008DF75F009EF124010EE75F009A425834D
:103A2B00F583E493900043F0900071A3E09008E0DD
:103A3B0075F009124010EE75F009A42583F583E4A7
:103A4B0093FD900044F09008E175F009EF124010DF
:103A5B00EE75F009A42583F583E493900045F0906F
:103A6B000071A3E09008E275F009124010EE75F0BA
:103A7B0009A42583F583E493900046F09008E37541
:103A8B00F009EF124010EE75F009A42583F583E4DD
:103A9B0093900047F0900071A3E09008E475F00953
:103AAB00124010EE75F009A42583F583E493900082
:103ABB0048F0ED6015900044E075F010A424CCF9AB
:103ACB00740835F0FA7BFF126124900045E0FF602B
:103ADB001175F010A424CCF9740835F0FA7BFF12A1
:0B3AEB006155900040E0900000F022C8
:10571D0090003B741FF090003C7407F090004974AA
:10572D003AF0E490004AF0900038E090004BF07BA6
:10573D00FF7A0D792A12612412614F7F0F121BB16E
:10574D00900005E0FF121B82900006E0FF121B8205
:0C575D007F1E121BB19000007432F0227D
:1035C100124C74D3900072E09400900071E094006A
:1035D100400A12611E90000074FAF022900071E01E
:1035E100FEA3E0FF9008F575F009124010EE75F0AA
:1035F10009A42583F583E493900040F09008F675C3
:10360100F009EF124010EE75F009A42583F583E46B
:1036110093900041F0900071A3E09008F775F009D4
:10362100124010EE75F009A42583F583E493900010
:1036310042F09008F875F009EF124010EE75F009AC
:10364100A42583F583E493900043F0900071A3E0F7
:103651009008F975F009124010EE75F009A4258360
:10366100F583E493FD900044F09008FA75F009EFBA
:10367100124010EE75F009A42583F583E4939000C0
:1036810045F0900071A3E09008FB75F0091240101D
:10369100EE75F009A42583F583E493900046F0903C
:1036A10008FC75F009EF124010EE75F009A42583AE
:1036B100F583E493900047F0900071A3E09008FD3A
:1036C10075F009124010EE75F009A42583F583E425
:1036D10093900048F0ED6015900044E075F010A45F
:1036E10024E5F9740835F0FA7BFF12612490004556
:1036F100E0FF601175F010A424E5F9740835F0FAC3
:0E3701007BFF126155900040E0900000F02226
:1057690090003B7424F090003C7407F09000497459
:105779003AF0E490004AF0900039E090004BF07B59
:10578900FF7A0D793A12612412614F7F0F121BB112
:10579900900005E0FF121B82900006E0FF121B82B9
:0C57A9007F1E121BB19000007432F02231
:10370F00124C74D3900072E09400900071E094001A
:10371F00400A12611E90000074FAF022900071E0CE
:10372F00FEA3E0FF90095F75F009124010EE75F0EF
:10373F0009A42583F583E493900040F09009607508
:10374F00F009EF124010EE75F009A42583F583E41C
:10375F0093900041F0900071A3E090096175F0091A
:10376F00124010EE75F009A42583F583E4939000C1
:10377F0042F090096275F009EF124010EE75F009F2
:10378F00A42583F583E493900043F0900071A3E0A8
:10379F0090096375F009124010EE75F009A42583A6
:1037AF00F583E493FD900044F090096475F009EF00
:1037BF00124010EE75F009A42583F583E493900071
:1037CF0045F0900071A3E090096575F00912401063
:1037DF00EE75F009A42583F583E493900046F090ED
:1037EF00096675F009EF124010EE75F009A42583F4
:1037FF00F583E493900047F0900071A3E090096780
:10380F0075F009124010EE75F009A42583F583E4D5
:10381F0093900048F0ED6015900044E075F010A40F
:10382F00244FF9740935F0FA7BFF1261249000459B
:10383F00E0FF601175F010A4244FF9740935F0FA08
:0E384F007BFF126155900040E0900000F022D7
:1057B50090003B7429F090003C7407F09000497408
:1057C5003AF0E490004AF090003AE090004BF07B0C
:1057D500FF7A0D794A12612412614F7F0D121BB1B8
:1057E500900005E0FF121B82900006E0FF121B826D
:0C57F5007F1E121BB19000007432F022E5
:10385D00124C74D3900072E09400900071E09400CB
:10386D00400A12611E90000074FAF022900071E07F
:10387D00FEA3E0FF9009C975F009124010EE75F036
:10388D0009A42583F583E493900040F09009CA754F
:10389D00F009EF124010EE75F009A42583F583E4CD
:1038AD0093900041F0900071A3E09009CB75F00961
:1038BD00124010EE75F009A42583F583E493900072
:1038CD0042F09009CC75F009EF124010EE75F00939
:1038DD00A42583F583E493900043F0900071A3E059
:1038ED009009CD75F009124010EE75F009A42583ED
:1038FD00F583E493FD900044F09009CE75F009EF47
:10390D00124010EE75F009A42583F583E493900021
:10391D0045F0900071A3E09009CF75F009124010A9
:10392D00EE75F009A42583F583E493900046F0909D
:10393D0009D075F009EF124010EE75F009A425833A
:10394D00F583E493900047F0900071A3E09009D1C6
:10395D0075F009124010EE75F009A42583F583E486
:10396D0093900048F0ED6015900044E075F010A4C0
:10397D0024B9F9740935F0FA7BFF126124900045E2
:10398D00E0FF601175F010A424B9F9740935F0FA4F
:0E399D007BFF126155900040E0900000F02288
:1061DF003022079000007401F02290003B742EF0E3
:1061EF0090003C7407F07BFF7A0D795A12612412EC
:0E61FF00614F7F1E121BB19000007432F0221F
:105ED000302807900000742FF02290000AE0643808
:105EE0006005A3E0B4390A12611E90000074FAF054
:105EF000227BFF7A0E790A12612490000AE0540F87
:095F0000F5489000007430F02215
:10592B0090000AE064386005A3E0B4390A12611EE6
:10593B0090000074FAF0227BFF7A0D796A126124D1
:10594B0090000AE0540FF548D202D20A9000C8E04A
:10595B00F527122BFE7BFF7A0E793A126124C202D5
:09596B00C20A90000074FEF02253
:10584D0090000AE0540FF548302002D200122C10BF
:10585D0030201B201304E53B70F9122C07C2007B8E
:10586D00FF7A0E793A12612490000074FEF0302117
:10587D0019201104E53B70F9122C077BFF7A0E7984
:0B588D003A12612490000074FEF0222B
:1053D400302356900001E0FF900034F0C223121BEA
:1053E40082900034E0FF1264FD5021900034E0FF0D
:1053F40090003CE02403F582E43400F583EFF09060
:10540400003CE004F0900000E004F022900034E05E
:10541400B42A079000007403F0227BFF7A0E791AF5
:0A54240012612490000074FAF022D7
:104F1F0030236A900001E0FF900034F0C223121B8F
:104F2F0082900034E0FFB42A0B90003BE090000029
:104F3F00F0D22822EFB4230B90003BE0900000F05A
:104F4F00C22822900034E0FF1264FD5021900034FB
:104F5F00E0FF90003CE02403F582E43400F583EF9A
:104F6F00F090003CE004F0900000E004F0227BFFA2
:0E4F7F007A0E791A12612490000074FAF02262
:105BE90030233F900001E0FF900034F0121B82C285
:105BF90023900034E0FFB42A0B90003BE0900000B2
:105C0900F0D22822EFB4230B90003BE0900000F083
:105C1900C228227BFF7A0E791A126124900000743F
:035C2900FAF0226C
:0A55DD00900043E0FF70033028380F
:1055E700121BB112637E1248208F5E900041E05279
:1055F7005EE55E60047F3180027F30121B823028B7
:1056070017C228E55E2430900023F0900033740120
:08561700F090000074F0F02295
:0F561F00900046E0FF121BB1900000E004F02263
:105B6100302340900001E0FF900034F0C223121B6B
:105B710082900034E0FFB42A079000007403F02201
:105B81001264FD500F900034E090000DF090000081
:105B9100E004F0227BFF7A0E791A12612490000052
:045BA10074FAF02280
:105FB100302332900001E0FF900034F0C223BF2A69
:105FC100079000007403F022900034E0B42307909E
:105FD1000000E004F0227BFF7A0E791A126124900E
:065FE100000074FAF0223A
:10542E0012637E900075EEF0A3EFF01248208F4FBE
:10543E0090003D7401F090000DE0B43108900041F1
:10544E00E0424F800E90000DE0B4301E900041E01F
:10545E00F4524F900075E0FEA3E0FFAD4F1247DF10
:10546E0012648290000074FEF0227BFF7A0E791A8D
:0A547E0012612490000074FAF0227D
:104BFF00900043E0FF7003302856121BB112637E02
:104C0F00900075EEF0A3EFF0E4F54F900041E0FF58
:104C1F00E54FC39F5027900075E475F001123FFADE
:104C2F00AFF0FE1248208F507423254FF582E434E5
:104C3F0000F583E550F0121B82054F80CE3028100F
:104C4F00C228E54F04900033F090000074F0F0227A
:104C5F0090003C740AF0900046E0FF121BB19000E8
:054C6F0000E004F0224A
:104B8600302375900001E0FF900034F0C223121B21
:104B960082900034E0FFB42A079000007403F022EC
:104BA600EFB42308900000E004F080391264FD5051
:104BB60038900034E0FF90003CE0FE04F074032ED1
:104BC600F582E43400F583EFF0900041E02409FF1C
:104BD600E433FE90003CE0D39FEE6480F874809846
:104BE6004016900000E004F0227BFF7A0E791A123C
:094BF600612490000074FAF02221
:105DAA00302337900001E0FF900034F0C223121B29
:105DBA0082900034E0FFB42A079000007403F022B6
:105DCA00EFB42307900000E004F0227BFF7A0E79FB
:0B5DDA001A12612490000074FAF022FD
:1054DF0012637E900075EEF0A3EFF090003C740A1B
:1054EF00F0E4F54F900041E0FFE54FC39F50279048
:1054FF000075E475F001123FFAAFF0FE90003CE04A
:10550F00FD04F074032DF582E43400F583E0FD1201
:10551F0047DF054F80CE7BFF7A0E793A12612490D8
:06552F00000074FEF022F2
:104EB00030236B900001E0FF900034F0C223121BFE
:104EC00082900034E0FFB42A079000007403F022BF
:104ED0001264FD501A900034E0FF90003CE0FE04A4
:104EE000F074032EF582E43400F583EFF080107B3C
:104EF000FF7A0E791A12612490000074FAF0229061
:104F00000041E02409FFE433FE90003CE0D39FEE33
:0F4F10006480F87480984006900000E004F0225E
:1043B500900043E0FF7006202803024460121BB101
:1043C50012637E900075EEF0A3EFF0124820121FE5
:1043D500E8900041E0B4011090006EE0FF121B82EE
:1043E50090006EE0900023F0900041E0B402209030
:1043F500006DE0FF121B8290006EE0FF121B8290A1
:10440500006DE0900023F090006EE0900024F090A5
:104415000041E06403703090006CE0FF121B829055
:10442500006DE0FF121B8290006EE0FF121B829070
:10443500006CE0900023F090006DE0900024F09077
:10444500006EE0900025F0302811C228900041E070
:10445500900033F090000074F0F022900046E0FFE9
:10446500121BB190003C740AF0900000E004F022A9
:1058010012203E5002803B1220168F4F900047E03D
:10581100FFE54FC39F402B900048E0FFE54FD39F2A
:10582100502012637E900075EEF0A3EFF0AD4F12A1
:1058310047DF7BFF7A0E793A12612490000074FEF3
:0C584100F02212611E90000074FAF022A8
:10562E0012203E5002803F1220168F4F900047E00E
:10563E00FFE54FC39F400B900048E0FFE54FD39F1F
:10564E004004E54F702012637E900075EEF0A3EFDC
:10565E00F0AD4F1247DF7BFF7A0E793A126124903C
:10566E00000074FEF02212611E90000074FAF02207
:104A1000900043E0FF700330285E121BB112637EEA
:104A2000900075EEF0A3EFF01248208F4F12490D61
:104A3000E4F54F746C254FF582E43400F583E0FF14
:104A40007423254FF582E43400F583EFF0746C2570
:104A50004FF582E43400F583E0FF121B82054FE539
:104A60004FC3940440CD30280FC228900033740304
:104A7000F090000074F0F022900046E0FF121BB1AD
:0D4A800090003C740AF0900000E004F02269
:105CEF007F0A1240428F4FE54F601212637E900081
:105CFF0075EEF0A3EFF0E54F14FD1247DFE54F7B94
:105D0F00FF600E7A0E793A12612490000074FEF053
:0F5D1F00227A0D79BA12612490000074FAF022F2
:1045E600900043E0FF7006202803024681121BB1AB
:1045F60012637E900075EEF0A3EFF0124820121FB2
:10460600E8900075E475F001123FFAAFF0FE12482B
:1046160020121FCC90006DE0FF900023F0A3F01253
:104626001B8290006EE0FF121B82900075E475F00D
:1046360001123FFAAFF0FE124820121FCC90006C18
:10464600E0FF900025F090006DE0900026F09000CD
:104656006EE0900027F0121B8290006DE0FF121BA7
:104666008290006EE0FF121B8230280FC228900055
:10467600337405F090000074F0F022900046E0FFDD
:10468600121BB190003C740AF0900000E004F02286
:1045340090000DE0540F75F00AA4FFA3E0540F2F70
:10454400F54F900010E0540F75F00AA4FF90000F8F
:10455400E0540F75F064A42FFF900011E0540F2F66
:10456400F550E54FC394014015E54FD39414500E14
:10457400E550C394014007E550D394FA400A126110
:104584001E90000074FAF02212637E900075EEF023
:10459400A3EFF0900075E475F001123FFAAFF0FE5E
:1045A400AD4F1247DF900010E0540F75F00AA4FFDE
:1045B40090000FE0540F75F064A42FFF900011E0F9
:1045C400540F2FF54F900075E0FEA3E0FFAD4F129E
:1045D40047DF7BFF7A0E793A12612490000074FE63
:0245E400F022C3
:103AF6007F0D124042EF701A900010E0B43010A310
:103B0600E0B4300BA3E0B43006A3E06430600302F7
:103B16003BE0900014E0FF64306004EFB4350E9093
:103B26000015E0540FD394054003023BE0900014C7
:103B3600E0FF64316004EFB43611900019E0B42060
:103B460007900018E0B42003023BE0900014E0FF69
:103B560064326004EFB43710900018E0B420079088
:103B66000017E0B420028072900014E0FF64336016
:103B760004EFB43809900015E0B42002805C900090
:103B860014E0FF64346005EF64397058900015E066
:103B9600540F75F00AA4FFA3E0540F2FF54F9000C1
:103BA60018E0540F75F00AA4FF900017E0540F7543
:103BB600F064A42FFF900019E0540F2FF550E54F45
:103BC600C394014015E54FD39414500EE550C394A9
:103BD600014007E550D394FA400A12611E90000096
:103BE60074FAF02212637E900075EEF0A3EFF09067
:103BF600003C740AF0E4F54F900041E0FFE54FC346
:103C06009F5027900075E475F001123FFAAFF0FE61
:103C160090003CE0FD04F074032DF582E43400F5D9
:103C260083E0FD1247DF054F80CE7BFF7A0E793A9F
:0A3C360012612490000074FEF022D9
:104B0A00900043E0FF700330285B121BB112637EF2
:104B1A00900075EEF0A3EFF0E4F54F900041E0FF4E
:104B2A00E54FC39F502C900075E475F001123FFACF
:104B3A00AFF0FE1248208F507423254FF582E434DB
:104B4A0000F583E550F07E00124820121B82054FC3
:104B5A0080C9302810C228E54F04900033F0900035
:104B6A000074F0F022900046E0FF121BB190003C66
:0C4B7A00740AF0D226900000E004F02243
:10506300302365900001E0FF900034F0C223BF2A93
:10507300079000007403F022900034E0FFB423088B
:10508300900000E004F0803DEF547FFF121B8290FC
:105093000034E0547FFF90003CE0FE04F074032EE4
:1050A300F582E43400F583EFF0900041E02409FF3A
:1050B300E433FE90003CE0D39FEE6480F874809864
:0950C3004006900000E004F02218
:1056CE0030234B900001E0FF900034F0C223BF2A3C
:1056DE00079000007403F022900034E0FFB4230B17
:1056EE00900000E004F0E004F080101264FD500F12
:1056FE00900034E090003EF0900000E004F0227B39
:0F570E00FF7A0E791A12612490000074FAF022CB
:104742002023030247DE900001E0FF900034F0C214
:1047520023BF2A079000007403F022900034E0FF88
:10476200B4230A900000E004F0E004F0221264FD99
:10477200505B90003EE0540F75F00AA4FF900034A5
:10478200E0540F2FF0E0900C8693FF900034F0126B
:104792001B82900034E0FF90003CE0FE04F07403C2
:1047A2002EF582E43400F583EFF0900041E0240915
:1047B200FFE433FE90003CE0D39FEE6480F8748007
:1047C20098900000E0400304F02214F0227BFF7A6C
:0D47D2000E791A12612490000074FAF02292
:1062E4003020099000DCE0F54D1263E1302203E434
:1062F400F54D30210B301E05754D0A8003754D2870
:07630400900000E004F0220C
:104FF900E54D7065124130900040E012401C502987
:1050090064502E6E502E78502E82502E8C5033962E
:105019005038A0503DAA5042B45047BE0000504AF3
:1050290012642C801C1261808017126698801212FB
:105039006699800D12669A800812669B8003126633
:105049009C30200F9000DEE09000A1F0900000E07D
:0A50590004F0229000007401F02220
:1064ED009000A1E070091263FB9000007401F0228E
:1053780030200D9000DCE0F54D1263E1E54D70FC46
:10538800302107754D05E54D70FCE4F54F30210CD3
:10539800126549121F971265A3121F9730200C122D
:1053A8006554121F971265A3121F97054FE54FC347
:1053B800940540D930200E9000DEE09000A1F090D6
:0C53C80000A1E070FA9000007401F022D7
:0166940022E3
:0166950022E2
:0166960022E1
:104A8D0030210A201E079000007401F02230200D05
:104A9D009000DCE0F54D1263E1E54D70FC3021072F
:104AAD00754D05E54D70FC30201B9000BFE0F52ADB
:104ABD00126554E4F54F121F97054FE54FC3940A45
:104ACD0040F41265A330211B9000C0E0F52A126559
:104ADD0049E4F54F121F97054FE54FC3940A40F473
:104AED001265A330200E9000DEE09000A1F0900042
:0D4AFD00A1E070FA121BE9E4900000F02225
:0166970022E0
:105C2C0030133E20233B9000A47464F0E542547F73
:105C3C00FF900A7D93900001F030260EE54230E78C
:105C4C0009EF900A8D93900001F0D223C2139000BB
:105C5C0001E0B42307900002E004F022E49000027B
:025C6C00F02224
:105C6E0030113E20233B9000A47464F0E540547F35
:105C7E00FF900A7D93900001F030260EE54030E74C
:105C8E0009EF900A8D93900001F0D223C21190007B
:105C9E0001E0B42307900002E004F022E490000239
:025CAE00F022E2
:10254C002024030226FE3023030226FE900002E024
:10255C00F552E4F09000A47464F012668B8F51D2A3
:10256C0023E551B430079000017430F022E551B4EA
:10257C0031079000017431F022E551B4320790001C
:10258C00017432F022E551B433079000017433F03A
:10259C0022E551B434079000017434F022E551B4B3
:1025AC0035079000017435F022E551B436079000E0
:1025BC00017436F022E551B437079000017437F0FE
:1025CC0022E551B438079000017438F022E551B47B
:1025DC0039079000017439F022E551B423109000B2
:1025EC00017423F0AF520552900002EFF022E55136
:1025FC00B42A07900001742AF022E551B4410790E7
:10260C0000017441F022E551B4420790000174427C
:10261C00F022E551B443079000017443F022E551D8
:10262C00B464079000017444F022202603C22322D4
:10263C00E551B461079000017461F022E551B46278
:10264C00079000017462F022E551B4630790000119
:10265C007463F022E551B464079000017464F022B5
:10266C00E551B465079000017465F022E551B4663C
:10267C00079000017466F022E551B46707900001E1
:10268C007467F022E551B468079000017468F02279
:10269C00E551B469079000017469F022E551B46A00
:1026AC0007900001746AF022E551B46B07900001A9
:1026BC00746BF022E551B46C07900001746CF0223D
:1026CC00E551B46D07900001746DF022E551B46EC4
:1026DC0007900001746EF022E551B46F0790000171
:1026EC00746FF022E551B470079000017470F02201
:0326FC00C22322D4
:0B6519007F209000037420F0A3DFFC43
:016524002254
:0F64FD00EFC394304007EFD39439500122C322EC
:104C740090000CE0FD6420602E90000BE0540F7552
:104C8400F00AA4FBAAF090000AE0540F75F064A4A3
:104C94002BFFE5F03AFEED540F7C002FFFEC3E9025
:104CA4000071F0A3EF803190000BE0FD64209000D0
:104CB4000A601AE0540F75F00AA4FFED540F7C004B
:104CC4002FFEEC35F0900071F0A3CE800BE0540F72
:104CD400FF900071E4F0A3EFF0E024FFF090007186
:054CE400E034FFF022A6
:10513400900009E0FD6420602B900008E0540F7596
:10514400F00AA4FBAAF0900007E0540F75F064A4E1
:105154002BFFE5F03AFEED540F7C002FFFEC3E9060
:105164000073802E900008E0FD6420900007601A10
:10517400E0540F75F00AA4FFED540F7C002FFEECF1
:1051840035F0900073F0A3CEF022E0540FFF9000AE
:0751940073E4F0A3EFF02229
:1063A100900005E0540F75F00AA4FFA3E0540F2FED
:1063B100900035F0D394004006E09415500122C3BB
:0163C10022B9
:10531B00E4FFEF75F003A4249DF582E4340AF583D2
:10532B00E493FE900004E0FDEE6D703BEF75F0032F
:10533B00A4249EF582E4340AF583E493FE900005E1
:10534B00E0FDEEB50521EF75F003A4249FF582E493
:10535B00340AF583E493FE900006E0FDEEB50507F5
:0C536B00900036EFF0D3220FBF33A7C331
:015377002213
:10525D00E4FF75F003EFA42436F582E5F0340BF589
:10526D0083E493FE900004E0FDEE6D703D75F00358
:10527D00EFA42437F582E5F0340BF583E493FE902B
:10528D000005E0FDEEB5052275F003EFA42438F519
:10529D0082E5F0340BF583E493FE900006E0FDEE1D
:0F52AD00B50507900037EFF0D3220FBF70A4C3F1
:0152BC0022CF
:1040420074032FF582E43400F583E0FD6431706976
:10405200FE74042FF582E43400F583E0FCEE75F083
:1040620003A4249DF582E4340AF583E4936C704240
:1040720074052FF582E43400F583E0FCEE75F0035D
:10408200A4249EF582E4340AF583E493B5042374F0
:10409200062FF582E43400F583E0FCEE75F003A40C
:1040A200249FF582E4340AF583E493B50404EE0414
:1040B200FF220EBE339B7F0022ED6432706DFE74D0
:1040C200042FF582E43400F583E0FD75F003EEA4DD
:1040D2002436F582E5F0340BF583E4936D70457474
:1040E200052FF582E43400F583E0FD75F003EEA4BC
:1040F2002437F582E5F0340BF583E493B505257496
:10410200062FF582E43400F583E0FD75F003EEA49A
:104112002438F582E5F0340BF583E493B50505EE1A
:0D4122002434FF220EBE70977F00227F0024
:01412F00226D
:10490D00EFC3943390006C50397431F0EF75F003B0
:10491D00A4249DF582E4340AF583E49390006DF0B0
:10492D00EF75F003A4249EF582E4340AF583E49335
:10493D0090006EF0EF75F003A4249FF582E4340A25
:10494D00803A7432F075F003EFA4249DF582E5F002
:10495D00340AF583E49390006DF075F003EFA42411
:10496D009EF582E5F0340AF583E49390006EF075C0
:10497D00F003EFA4249FF582E5F0340AF583E49368
:05498D0090006FF02214
:10644300900005E0540F75F00AA4FFA3E0540F2F4A
:05645300900038F0226A
:10645800900005E0540F75F00AA4FFA3E0540F2F35
:05646800900039F02254
:10646D00900005E0540F75F00AA4FFA3E0540F2F20
:05647D0090003AF0223E
:10637E0090004BE0FF90004AE08FF0A4FF900049A0
:10638E00E07C002FFFEC35F0FE900042E02FFFEC9A
:03639E003EFE229E
:10648200900044E075F010A4244DF9740235F0FA3E
:056492007BFF026155D3
:03668B007F032268
:10642C00302008900023E0FF1265313021089000E5
:07643C0023E0FF1265252299
:10618000E4F55E900033E0FFE55EC39F5021742389
:10619000255EF582E43400F583E0F55F302004FFEE
:0F61A000126531302105AF5F126525055E80D491
:0161AF0022CD
:0166980022DF
:0166990022DE
:01669A0022DD
:01669B0022DC
:01669C0022DB
:0C65250012655F121F971265AA021F97F3
:0C65310012656A121F971265AA021F97DC
:10413000E4F55EF55FF560900072E02401FF900009
:1041400071E03400FEC3EF940AEE94005005A3E042
:1041500004F560D3EF9463EE9400404C900072E05D
:104160002401FB900071E03400FA7C007D64AF0311
:10417000FE123FA58F5EEF75F064A4FFC3EB9FFFB7
:10418000EA95F0FE7C007D0A123FA58F5FA3E00454
:10419000FFE55E75F064A4FEC3EF9EFFE55F75F07A
:1041A0000AA4FEC3EF9EF560900072E02401FF9028
:1041B0000071E03400FED3EF9409EE940040197CC6
:1041C000007D0A123FA58F5FA3E004FFE55F75F055
:1041D0000AA4FEC3EF9EF5607430255EF55E743070
:1041E000255FF55F74302560F560302014AF5E12F6
:1041F0006531AF5F126531AF601265317F2A12659C
:1042000031302114AF5E126525AF5F126525AF60B6
:084210001265257F2A126525C5
:014218002283
:06611E007BFF7A0D798A77
:066124008B5F8A608961B7
:10612A007F01121BB1E4F562AB5FAA60A9618562C7
:10613A0082758300123F66FF121B820562E562C305
:04614A00941040E489
:01614E00222E
:06614F007BFF7A0D79DAF6
:066155008B608A61896283
:10615B007F11121BB1E4F563AB60AA61A962856381
:10616B0082758300123F66FF121B820563E563C3D2
:04617B00941040E458
:01617F0022FD
:105D2E007BFF7A0E794A126155125E96E4F55EF5A6
:105D3E005FE55F900A3C93FDAF5FAE5E1247DFE515
:105D4E005F900A3C93FDAF5FAE5E125974055FE53E
:0E5D5E005F7002055EC3943AE55E940040D388
:015D6C002214
:01669D0022DA
:01669E0022D9
:01669F0022D8
:0166A00022D7
:0166A10022D6
:0166A20022D5
:0166A30022D4
:10630B007BFF7A0E79CA126124125D2E12669D12E2
:10631B00669E12669F1266A01266A11266A2126694
:07632B00A3121BCB021BDAD9
:1061B000755E01755F007560B3E4F561AF617E00E7
:1061C000124820AB5E0560E560AA5F7002055F14AF
:0E61D000F9EF123F930561E561C3943A40DE9A
:0161DE00229E
:10629300125E96E4F55EF55FAF5FAE5E124820AD29
:1062A30007AF5FAE5E125974055FE55F7002055E6E
:0962B300C3943AE55E940040DF5B
:0162BC0022BF
:10633200E4F564F565AF65AE6412620DAD07AF6555
:10634200AE641247DF0565E56570020564C3943AE1
:06635200E564940040DF49
:016358002222
:105F0900755E01755F007560B3E4F561F562AF62B6
:105F1900AE6112620DAB5E0560E560AA5F700205B5
:105F29005F14F9EF123F930562E56270020561C3E0
:085F3900943AE561940040D6A2
:015F4100223D
:105F4200755E01755F007560B3E4F561F562AB5E85
:105F52000560E560AA5F7002055F14F9123F4DFD0E
:105F6200AF62AE611247DF0562E56270020561C38E
:085F7200943AE561940040D669
:015F7A002204
:1047DF00C2B0758400D2C2C2C6D2C6C2C4D2C5C2CC
:1047EF00C330C3FD74A0F5C2C2C5C2C330C3FD8EB2
:1047FF00C2C2C330C3FD8FC2C2C330C3FD8DC2C29C
:10480F00C330C3FDD2C4C2C320C4FD121F7FD2B0B8
:10481F0022758400C2C3D2C530C3FD74A0F5C2C2D5
:10482F00C5C2C330C3FD8EC2C2C330C3FD8FC2C267
:10483F00C330C3FDC2C4D2C5C2C330C3FD74A1F51A
:10484F00C2C2C5C2C330C3FDC2C2C2C330C3FD851D
:10485F00C207D2C4C2C320C4FD22D2C2C2C6D2C6AE
:08486F00D2C4C2C320C4FD2223
:102BFE00754700122C1950FB22754700122CA2505B
:102C0E00FB22754700122C5950FB22758400E547B4
:102C1E0075F003A4902C2673022CBE022CCD022C30
:102C2E00EB022CD4022CF7022CFE022D06022CCD28
:102C3E00022D14022CD4022D24022D2D022CBE02A4
:102C4E002CCD022D3B022CD4022D47758400E54776
:102C5E0075F003A4902C6673022CBE022CCD022CB0
:102C6E00EB022CD4022CF7022CFE022CBE022CCD31
:102C7E00022CEB022CD4022CF7022CFE022CF702B3
:102C8E002CFE022D06022CCD022D49022CD4022D33
:102C9E0024022D47758400E54775F003A4902CAFF0
:102CAE0073022CBE022CCD022D3B022CD4022D47DA
:102CBE00C2FA122D59122D59759B000547C32230A9
:102CCE00F9020547C32230F912E59A20E7FB122DCF
:102CDE0059D2FA122D59122D590547C322C2FA1292
:102CEE002D59759B040547C322753A1E0547C3220D
:102CFE00E53A70020547C322C2FA122D59122D7AF7
:102D0E00F59B0547C322C2FA122D59122D8944078D
:102D1E00F59B0547C322122D6BF53B0547C3227564
:102D2E00840F30DE04E53B70020547C322C2FA125F
:102D3E002D59759B080547C322D322C2FA122D596D
:092D4E00122D894405F59B05478F
:102D5700C322000000000000000000000000000087
:102D670000000022902D72E54893225A5A5A5A5A67
:102D7700FAFAFA902D81E548932200B45AE12D879B
:102D87007ADB902D90E54893220000000000008038
:012D970080BB
:105BA5002A2A3132333435362A2A2A2A31323334F5
:105BB50035302A2A44313233343536373839302AAC
:105BC50023414243202056455253494F4E20322E01
:105BD50031302020202020205349454D454E53206B
:045BE500202020203C
:10469600302920C229E542540F905BB99390008CD3
:1046A600F0786876329000B4E0601512601C125EF5
:1046B60020800D7868E67008900078F0900089F008
:1046C600302A40C22AE540540F905BB99390008B84
:1046D600F0754A321259BD301E06740044B3700993
:1046E600201E099000B5E06003125DE5301E0674D9
:1046F6000044B37003201E03125FE7201E151260EC
:10470600BA8010E54A700C900079F0900088F0901D
:1047160000EDF03025199000B6E0601F754B32129F
:10472600668E90007CEFF0C225125E5B026051E55A
:0C4736004B700890007AF090008AF0228E
:105FE700900079E0FF04F0EF905BA593FF90008BA2
:105FF700E0FEEF6E6011EEB42A089000797401F0AC
:106007008005E4900079F0900079E0B40A06E4F0A6
:05601700D221D22B2272
:10601C00900078E0FF04F0EF905BA593FF90008C6C
:10602C00E0FEEF6E6011EEB42A089000787401F077
:10603C008005E4900078F0900078E0B40A06E4F073
:05604C00D220D22B223E
:1060510090007AE0FF04F0EF905BA593FF90007C45
:10606100E0FEEF6E6011EEB42A0890007A7401F040
:106071008005E490007AF090007AE0B40A06E4F03A
:05608100D222D22B2207
:105DE500900088E0FF04F0747F2FF582E43400F51D
:105DF50083E0FF90008BE0FEEF6E6011EEB42308A8
:105E05009000887401F08005E4900088F090008887
:0B5E1500E0B40906E4F0D221D21F2205
:105E2000900089E0FF04F0747F2FF582E43400F5E0
:105E300083E0FF90008CE0FEEF6E6011EEB423086B
:105E40009000897401F08005E4900089F090008949
:0B5E5000E0B40906E4F0D220D21F22CB
:105E5B0090008AE0FF04F0747F2FF582E43400F5A4
:105E6B0083E0FF90007CE0FEEF6E6011EEB4230840
:105E7B0090008A7401F08005E490008AF090008A0B
:0B5E8B00E0B40906E4F0D222D21F228E
:1060BA0090007BE0FF04F0EF905BAF93FF90008BC2
:1060CA00E0FEEF6E6011EEB42A0890007B7401F0D6
:1060DA008005E490007BF090007BE0B40A04E4F0D1
:0360EA00D22C2293
:10623B0090007F7423F0A3F0E4FF74B72FF582E492
:10624B003400F583E0FE74812FF582E43400F5838E
:0C625B00EEF00FBF06E49000877423F003
:016267002214
:10567E00121ADF121BCB7F01121BB17BFF7A5B79F3
:10568E00D91261247BFF7A5B79C912615575391481
:10569E00E490007EF090007DF0FF744C2FF582E4D4
:1056AE003400F583E4F0745C2FF582E43400F58366
:1056BE00E4F00FBF10E4E53970FC121BCB021BDACD
:104E3F0090007EE0FFD3940F501FEF04FF121BB1C1
:104E4F0090008BE0FF90007EE0FE04F0744C2EF596
:104E5F0082E43400F583EF80437F01121BB1E4F548
:104E6F005E744D255EF582E43400F583E0FF744CEB
:104E7F00255EF582E43400F583EFF0744C255EF582
:104E8F0082E43400F583E0FF121B82055EE55EC30A
:104E9F00940F40CD90008BE0FF90005BF0121B82CF
:014EAF0022E0
:104D5C0090007DE0FFD3940F5020EF2411FF121B25
:104D6C00B190008CE0FF90007DE0FE04F0745C2EAE
:104D7C00F582E43400F583EF80437F11121BB1E41C
:104D8C00F55E745D255EF582E43400F583E0FF7416
:104D9C005C255EF582E43400F583EFF0745C255EEF
:104DAC00F582E43400F583E0FF121B82055EE55EBC
:104DBC00C3940F40CD90008CE0FF90006BF0121B61
:014DCC008264
:014DCD0022C3
:03668E007F012267
:1059BD009000EDE0FF700E90008BE0B42A07900090
:1059CD00ED7401F022EFB4011390008BE0B42307C6
:1059DD009000ED7402F022E49000EDF09000EDE007
:1059ED00B4021490008BE0B430089000EE7401F016
:0859FD008000E49000EDF022AF
:10421900E53760021537E53A6002153A900093E0F8
:10422900600214F0900097E0600214F090009BE0A7
:10423900600214F090009FE0600214F09000A2E088
:10424900600214F09000AAE0600214F09000B2E05D
:10425900600214F022E538600215389000A1E06090
:104269000214F0900092E0600214F0900096E06071
:104279000214F09000A7E0600214F022E539600210
:104289001539E53B6002153BE54C6002154CE54DDF
:104299006002154D7868E6600116E54A6002154A24
:1042A900E54B6002154B9000AFE0600214F09000FE
:1042B9009AE0600214F090009EE0600214F0900011
:1042C900A8E0600214F09000EFE0600214F02222EE
:1042D9009000A4E0600214F0229000A3E0600214B0
:0242E900F022C1
:1026FF00202046554E4354494F4E2031382020203C
:10270F0000202020454D455247454E43592020205B
:10271F002000202020205354414E44425920202095
:10272F002020524144494F204F524947494E41546E
:10273F00452054454C434F204F524947494E415431
:10274F00452020202046554E4354494F4E203120DE
:10275F00202020202046554E4354494F4E203220F2
:10276F00202020202046554E4354494F4E203320E1
:10277F00202020202046554E4354494F4E203420D0
:10278F00202020202046554E4354494F4E203520BF
:10279F00202020202046554E4354494F4E203620AE
:1027AF00202020202046554E4354494F4E2037209D
:1027BF00202020202046554E4354494F4E2038208C
:1027CF00202020202046554E4354494F4E2039207B
:1027DF002020202052454345495645204D4F444522
:1027EF002020205452414E534D4954204D4F4445C3
:1027FF002020202046554E4354494F4E2031302043
:10280F002020202046554E4354494F4E2031312031
:10281F002020202046554E4354494F4E2031322020
:10282F002020202046554E4354494F4E203133200F
:10283F002020202046554E4354494F4E20313420FE
:10284F002020202046554E4354494F4E20313520ED
:10285F002020202046554E4354494F4E20313620DC
:10286F002020202046554E4354494F4E20313720CB
:10287F002020202046554E4354494F4E20313820BA
:10288F0020203A0036AA340031552EAA2C002955A3
:0E289F0026AB240021551EAB1C001955140059
:102354009000E8E0700302254B202D0F9000B0E0C0
:1023640060099000AFE07003022547202D03022589
:102374004BC22D9000B0E0FF701CE540B40B0C90F4
:1023840000AF7414F09000B0E004F0E540640C6019
:102394000302254B8015EF640160030224A6E54087
:1023A400B40B030224B6E540B40C0D9000AF7414D2
:1023B400F09000B07403F0229000DBE0C39403506B
:1023C4002EE54094004028E54094085022E540144E
:1023D4009000ACF09000AE7401F09000ACE075F0A9
:1023E40010A42451F9742735F0FA7BFF126124906C
:1023F40000DBE0B4032FE540D394074028E5409484
:102404000A5022E540149000ACF09000AE7401F044
:102414009000ACE075F010A42451F9742735F0FA5B
:102424007BFF1261249000DBE064047035E54064B6
:1024340008702F7BFF7A2779C11261247BFF7A27EA
:1024440079F11261559000EBE0B403031265B19089
:1024540000ECE0B403031265BD1263E19000B174B3
:1024640001F09000DBE064047034E5406409702EF0
:102474007BFF7A2779D11261247BFF7A2779E112D5
:1024840061559000EBE0B403031265B79000ECE0F3
:10249400B403031265C31263FBE49000B1F0E402D9
:1024A40025479000B0E06403600302254BE540B487
:1024B4000C079000AF7414F022E540B40B0D9000AB
:1024C400AF7414F09000B07401F022E540B4092D0B
:1024D4009000ACE09000ADF09000AC7414F0E49087
:1024E40000ABF09000AE04F07BFF7A2679FF126116
:1024F400247BFF7A277910126155E480469000DB33
:10250400E0C394035007E540C394084005E540B494
:102514000A30E540B40A089000AC7409F08008E57C
:102524004024099000ACF09000AE7401F09000AC2F
:10253400E075F010A42471F9742735F0FA7BFF12CA
:082544006124E49000B0F022D4
:1017D5009000DBE064047003021ADE9000AEE07056
:1017E50003021ADE1266559000ABE0FF702A9000E6
:1017F500ACE0FE6407600BEE64146006EEC394056E
:1018050050079000AB7401F022EE9000ABB40804D1
:101815007408F0227404F022EFB401030219209039
:1018250000ABE06402707B9000AAE06003021ADE60
:101835009000ACE0FF6003B4070C902895E493F5A5
:1018450016740193F517EFB4010C902897E493F5FE
:1018550016740193F517EFB4020C9028A1E493F5E3
:1018650016740193F517EFB4030C9028A3E493F5D0
:1018750016740193F517EFB4040C90289DE493F5C5
:1018850016740193F517EFB4140C902893E493F5AF
:1018950016740193F5179000C4E0F52812665B02F3
:1018A50019FF9000ABE06403706A9000AAE0600342
:1018B500021ADE90289193F516740193F51790009E
:1018C500C5E0F52812665B9000B17401F012663729
:1018D500E49000ABF09000AEF09000ACE0641460D2
:1018E50003021ADE9000ADE09000ACF012665E12C5
:1018F5001BCBE49000B1F090009CF0900099F09023
:1019050000DEE0FF9000D9E02F9000A1F09000A547
:10191500740AF0229000ABE0B40420902891E4937F
:10192500F516740193F5179000C6E0F52812665B6D
:101935001266559000AA7478021A909000ABE0FFE9
:1019450064056003021A079000AAE06003021ADE2C
:101955009000ACE0FEB4050C9028A5E493F5167450
:101965000193F517EEB4060C9028A7E493F51674C9
:101975000193F517EEB4090C9028A5E493F51674B8
:101985000193F517EEB40A0C9028A5E493F51674A7
:101995000193F517EEB40B0C9028A5E493F5167496
:1019A5000193F517EEB40C0C9028A5E493F5167485
:1019B5000193F517EEB40D0C9028A7E493F5167472
:1019C5000193F517EEB40E0C9028A7E493F5167461
:1019D5000193F517EEB40F0C9028A7E493F5167450
:1019E5000193F517EEB4100C9028A7E493F516743F
:1019F5000193F5179000C4E0F5289000AA74280219
:101A05001A90EF64066003021A989000AAE060033A
:101A1500021ADE9000ACE0FF64056004EFB4060C2A
:101A2500902895E493F516740193F517EF64096012
:101A350004EFB40D0C902897E493F516740193F513
:101A450017EF640A6004EFB40E0C9028A1E493F537
:101A550016740193F517EF640B6004EFB40F0C9047
:101A650028A3E493F516740193F517EF640C60044D
:101A7500EFB4100C90289DE493F516740193F517B7
:101A85009000C4E0F5289000AA7428F09000ABE01F
:101A950004F0229000ABE0FFB407279000AAE070A5
:101AA5003890289193F516740193F5179000C5E0C9
:101AB500F5289000B17401F0E49000ABF09000AE11
:101AC500F022EFB4081312665E126658E49000AB7C
:0A1AD500F09000AEF09000B1F02296
:101F5300000000000000000000000000000022C09C
:101F630000C001790478B4D8FED9FAD001D0002298
:101F7300C0007814121F62D8FBD00022C0E075376E
:101F830005E53770FCD0E022C0E075370FE5377008
:101F9300FCD0E022C0E0753764E53770FCD0E02266
:101FA300A42582F582E58335F0F58322B40A002265
:101FB300C0E0C3997001D3D0E022B50601225007D7
:101FC300B5070122400122D322EF75F06484243047
:101FD30090006CF0E5F0A375F00A842430F0A3E5DB
:101FE300F02430F022EF75F06484243090006CF01C
:101FF300E5F0A375F00A842430F0A3E5F02430F073
:1020030090006CE0B4300B7420F0A3E0B4300374A0
:1020130020F02290000DE0540FFFA3E0B4200280D3
:1020230019540FCF75F00AA42FFFA3E0B420028048
:1020330009540FCF75F00AA42FFF22C006C005C0B4
:082043000490000DE0540FFFB2
:10204B00FEA3E0B42003C3802C540FFDCF75F00A20
:10205B00A42FFFA3E0B42003C3801A540FFCEE752A
:10206B00F064A420D20EFEED75F00AA42E40052CD0
:10207B0040028001D3D004D005D0062275F06484D1
:10208B00F6E5F00875F00A84F608A6F00822C00100
:10209B007900E6B4FF028027F908E6B4FF03C3809A
:1020AB0022E975F00AA426F908E6B4FF03C38013EE
:1020BB00E975F00AA420D207C3264003F98004D3A4
:1020CB00D00122E9D00122E675F00AA40826227875
:1020DB0047EE1220877545007546007849902133ED
:1020EB007908EF134007A3A3A3A3A3801CC0E0C0F0
:1020FB0000C001C37905E49336D4A2E4540FF6A3D0
:10210B0018D9F3D001D000D0E0D9D8E545600C75D3
:10211B004609754709754809754909854645854737
:10212B0046854847854948220605020000020105FD
:10213B00000004020001000804000200060900046C
:10214B000002090108000408030601080607020340
:101D290020205455524E204F4E205357202020201A
:101D39000020205455524E204F464620535720200C
:101D4900200044313233343536373839302A23418B
:101D5900424302AB055508000AAB0D55100012AB02
:101D6900155518001AAB1D55200022AB2555280022
:101D79002AAB2D55300032AA3555202054455354ED
:101D890020524F5554494E45202020205645525344
:101D9900494F4E20312E302020202054455354499C
:101DA9004E4720454550524F4D202020544553540D
:101DB900494E4720564F49434520205445535449DD
:101DC9004E472044544D4620312020544553544910
:101DD9004E472044544D4620322020205445535428
:101DE900494E472052533233322020205445535410
:101DF900494E47205253343835202020205445532A
:101E090054494E47205054542020205445535420BF
:101E19004155582052454C4159202054455354208E
:101E290043542052454C4159202020544553494E92
:101E3900472052494E47494E472020202020202044
:101E490020202020202020202020205445535420C9
:101E59004C494E452052414C415954455354204C0C
:101E6900494E452053454E53452B54455354204C18
:101E7900494E452053454E53452D20205445535432
:101E8900204449475F494E2020202054455354207F
:101E9900494E50555420564F4C54205445535420C4
:101EA9004C494E452052454C415954455354205AAA
:101EB90045524F2043524F53532054455354494E92
:101EC9004720535155454C434820202054455354ED
:101ED900494E47204850462020202054455354203D
:101EE90054454C434F20564F5820205445535420B5
:101EF900524144494F20564F5820205445535420AD
:101F0900454D5F4F50545020202020202020202074
:101F190020202020202020202020202020202020B8
:101F290020202020202020202020205445535420E8
:101F3900434F4D504C45544544202020205445538F
:0A1F490054204641494C4544202035
:100EDA007BFF7A1D79831261247BFF7A1D79931235
:100EEA00615512658B7BFF7A1D79A3126124121B4F
:100EFA00DA12658B7F007E001248208F4F7DAA7F11
:100F0A00007E001247DF7F007E00124820EF64AAAD
:100F1A00600C7BFF7A1F79431261551266917D55E9
:100F2A007F007E001247DF7F007E00124820EF64B8
:100F3A0055600C7BFF7A1F7943126155126691AD99
:100F4A004F7F007E001247DF7BFF7A1F79331261E1
:100F5A002412658B7BFF7A1D79B31261241265CF47
:100F6A00126549754700754801753914122C10E548
:100F7A003970FC122C0712660B754700754801750B
:100F8A003905E53970FCD202D20A122BFEC202C21E
:100F9A000A7BFF7A1F793312612412658B7BFF7AF1
:100FAA001D79C3126124121BDA12658B7F31126517
:100FBA006A753932E53970FC1265AA3013FD12657B
:100FCA00AAE542547FFFEF901D4B93FFEFB4310E19
:100FDA007BFF7A1F793312612412658B800C7BFFA9
:100FEA007A1F79431261551266917BFF7A1D79D374
:100FFA00126124121BDA12658B7F3112655F12654A
:10100A00931265AA3011FDE540547FFFEF901D4B06
:10101A0093FFEFB4310E7BFF7A1F793312612412EA
:10102A00658B800C7BFF7A1F79431261551266919A
:10103A007BFF7A1D79E3126124121BDA12658B7524
:10104A008400759850C299C2987599433098FD7575
:10105A008400E5996443600C7BFF7A1F794312612F
:10106A00551266917BFF7A1F793312612412658BC0
:10107A007BFF7A1D79F3126124121BDA12658B1237
:10108A006613758400759850C299C2987599433051
:10109A0099FD7BFF7A1F793312612412658B7BFFDE
:1010AA007A1E7903126124121BDA12658B1263E12C
:1010BA00126593E53ED39432400C7BFF7A1F794345
:1010CA001261551266911263FB126593E53EC39451
:1010DA00AA500C7BFF7A1F79431261551266917BE5
:1010EA00FF7A1F793312612412658B7BFF7A1E798E
:1010FA0013126124121BDA12658B1265B112659301
:10110A00E53DD3940A400C7BFF7A1F79431261555F
:10111A001266911265B7126593E53DC394AA500C05
:10112A007BFF7A1F79431261551266917BFF7A1F02
:10113A00793312612412658B7BFF7A1E792312613F
:10114A0024121BDA12658B1265BD12658B12658B30
:10115A001265C37BFF7A1F793312612412658B7B78
:10116A00FF7A1E7953126124121BDA12658B1265FB
:10117A00C912658B12658B1265CF12658B12658B4E
:10118A007BFF7A1E7983126124121BDA12658B3077
:10119A00DC1D7BFF7A1D792912615520DCFD121BAB
:1011AA00DA7BFF7A1F793312612412658B801B7BED
:1011BA00FF7A1D793A12615530DCFD121BDA7BFF8A
:1011CA007A1F793312612412658B7BFF7A1F7903A8
:1011DA00126124121BDA12658B1265F3501F7BFF12
:1011EA007A1D79291261551265F340FB121BDA7BCD
:1011FA00FF7A1F793312612412658B801D7BFF7A77
:10120A001D793A1261551265F350FB121BDA7BFF06
:10121A007A1F793312612412658B7BFF7A1E7993C8
:10122A00126124121BDA12658BE53CC3940A40074B
:10123A00E53CD39446400C7BFF7A1F7943126155F3
:10124A001266917BFF7A1F793312612412658B7BB8
:10125A00FF7A1E79B3126124121BDA12658B1265AA
:10126A007512662E40FB12662E50FB12662E40FB4C
:10127A007BFF7A1F793312612412658B1265A37B77
:10128A00FF7A1E79C3126124121BDA12658B12656A
:10129A00D5400F1263E11263FB1265D550F5800247
:1012AA0080F17BFF7A1F793312612412658B7BFFF1
:1012BA007A1E79F3126124121BDA12658B12658089
:1012CA001265DB50FB800280F71265A37BFF7A1F51
:1012DA00793312612412658B7BFF7A1E79D31261EE
:1012EA0024121BDA12658B12657512659B901D5DBF
:1012FA00E493F508740193F50912659B901D5FE468
:10130A0093F508740193F50912659B901D61E493A6
:10131A00F508740193F50912659B901D63E493F532
:10132A0008740193F50912659B901D65E493F5080D
:10133A00740193F50912659B901D67E493F508748F
:10134A000193F50912659B901D69E493F5087401F0
:10135A0093F50912659B901D6BE493F5087401934C
:10136A00F50912659B901D6DE493F508740193F5D8
:10137A000912659B901D6FE493F508740193F509B2
:10138A0012659B901D71E493F508740193F5091297
:10139A00659B901D73E493F508740193F509126532
:1013AA009B901D75E493F508740193F50912659BEA
:1013BA00901D77E493F508740193F50912659B90E3
:1013CA001D79E493F508740193F50912659B901D44
:1013DA007BE493F508740193F50912659B901D7DD2
:1013EA00E493F508740193F50912659B901D7FE457
:1013FA0093F508740193F50912659B901D81E49396
:10140A00F508740193F5091265A37BFF7A1F7933F6
:09141A0012612412658B0212F12B
:0114230022A6
:08658B0075390AE53970FC22A4
:08659300753902E53970FC22A4
:08659B00753905E53970FC2299
:0366910080FE2266
:080003000228AD00000000001E
:08000B000228AE000000000015
:080013000229E10000000000D9
:08001B003200000000000000AB
:09002300320000000000000000A2
:08002B000228B10000000000F2
:08003300320000000000000093
:0A003B003200000000000000000089
:0900430032000000000000000082
:08004B0032000000000000007B
:08005300320000000000000073
:08005B0002291300000000005F
:08006300320000000000000063
:08006B00022932000000000030
:080073000228B70000000000A4
:08007B000229E2000000000070
:0800830002291000000000003A
:08008B0032000000000000003B
:10009300022A000000000000000000000000000031
:1000A3003275FF0775FFDE75FFAD75840F75E107C8
:1000B30075E20475E34475840F75A43575A5097558
:1000C300A6FF75A7FF759CFF759D00759E00759F24
:1000D300F075D8FF75E8FF75F80F75AD0F758401DE
:1000E30075893075888F75840275893075888F7529
:1000F300840F758A80758C67780874FF0000000090
:100103000000000000000000D5E0F1D8EDE58C30E0
:10011300E7FB759701758A0043890475840075B7F9
:100123001075840F438901758D01758F01758E02DA
:100133007480D5E0FD438902E58930E4FB759702BD
:1001430075840075D10775840075BB0175BA007598
:10015300BCF075C70075C60075C5FF75C4FF75E8AB
:100163008175840275BB0475BA0075BCF175C60050
:1001730075C4FF75E88875840075D484758401752A
:10018300D484758400C2F8759A47759D1A43F8099B
:1001930075870075840075B90075A90075910075A0
:1001A300985075840175981075840075C04075C3A7
:1001B3000075CFC9758400758E0075892075880513
:1001C300758400758A00758B6F758CF4758D6F431C
:1001D300885075840075C90075CA0075CB0075CC4D
:1001E3000075CD0075840175C91875CA8075CBFB80
:1001F30075CDFB75CC80D2CA75840275C91875CAD2
:10020300A675CBAF75CDAF75CCA6D2CA7584007574
:10021300A8AF75B80075E6A475E71775F60075F70E
:10022300019000007F007E20E4F0A3DFFCDEFA757E
:0202330027FFA3
:100235007528FF7529FF752AFF752BFF752CFF752E
:080245002DFFD2B61248692218
:10597400AC84A2AF922EABB1C2AF75840F53A1FE1B
:1059840075B121E4F58443B701F584438F01786C44
:10599400768008F6EF26F618EE36F6E6FE08E6F50B
:1059A400828E83EDF0E4F584538FFEF58453B7FEC5
:0859B4008BB18C84A22E92AF8E
:0159BC0022C8
:10620D00AD84A2AF922EACB1C2AF75B121756680CF
:10621D00756700EF2567F567EE3566F5668567826C
:0D622D00F583E493FF8CB18D84A22E92AF17
:01623A002241
:105E9600AF84A2AF922EAEB1C2AF786C7680087690
:105EA6000075B121E4F58443B701F584758F0318B5
:105EB600E6FC08E6F5828C83E4F0F58FF58453B7AB
:095EC600FE8EB18F84A22E92AF72
:015ECF0022B0
:0300000002653D59
:0C653D00787FE4F6D8FD75816D0242EB1A
:103F4D00BB010689828A83E0225002E722BBFE0272
:093F5D00E32289828A83E49322A5
:103F6600BB010CE58229F582E5833AF583E0225010
:103F760006E92582F8E622BBFE06E92582F8E2225A
:0D3F8600E58229F582E5833AF583E4932274
:103F9300BB010689828A83F0225002F722BBFE010D
:023FA300F32207
:103FA500BC000BBE0029EF8DF084FFADF022E4CC00
:103FB500F875F008EF2FFFEE33FEEC33FCEE9DECC9
:103FC500984005FCEE9DFE0FD5F0E9E4CEFD22ED0F
:103FD500F8F5F0EE8420D21CFEADF075F008EF2F59
:103FE500FFED33FD4007985006D5F0F222C398FD4A
:053FF5000FD5F0EA22E7
:103FFA00A3F8E0C5F025F0F0E5821582700215837A
:06400A00E0C838F0E822D6
:0C401000A42582F582E5F03583F58322BB
:10401C00D083D082F8E4937012740193700DA3A333
:10402C0093F8740193F5828883E473740293686047
:06403C00EFA3A3A380DF47
:00000001FF
